:100000000C9446000C9463000C9463000C94630001
:100010000C9463000C9463000C9463000C946300D4
:100020000C9463000C9463000C9463000C946300C4
:100030000C9463000C9463000C9463000C946300B4
:100040000C9463000C9463000C9463000C946300A4
:100050000C9463000C9463000C9463000C94630094
:100060000C9463000C9463000C9463000C94630084
:100070000C9463000C9463000C9463000C94630074
:100080000C9463000C9463000C94630011241FBE55
:10009000CFEFD0E1DEBFCDBF11E0A0E0B1E0ECE6F4
:1000A000FFE000E00BBF02C007900D92A830B1073F
:1000B000D9F711E0A8E0B1E001C01D92A830B10766
:1000C000E1F70C947D000C940000F8948FEF8ABB4C
:1000D0008BBB78940895CF930E946500C1E04FEFE9
:1000E00060E08C2F0E94310160E070E088EC92E4C7
:1000F0000E94DB00CC0F99F7F1CFCFEFD0E1DEBF4C
:10010000CDBF0E946B0080E090E00C94B5079F92F9
:10011000AF92BF92CF92DF92EF92FF920F931F9315
:10012000CF935B016C0120E030E040E452E40E9498
:100130000504DC01CB01BC01CD010E943601DC01CC
:10014000CB01982EC0E0C81758F52BEA3AEA4AEAE4
:1001500050E4C601B5010E94EA027B018C0120E057
:1001600030E040E85FE30E942105882314F481E039
:1001700012C020E030E04FE753E4C801B7010E940D
:10018000B504181614F480E006C0C801B7010E9437
:100190003601DC01CB018A95F1F7CF5FC915A8F2D2
:1001A000CF911F910F91FF90EF90DF90CF90BF9074
:1001B000AF909F9008959F92AF92BF92CF92DF929F
:1001C000EF92FF920F931F93CF935B016C0120E09E
:1001D00030E040E85DE30E94EA02DC01CB01BC01B3
:1001E000CD010E943601DC01CB01982EC0E0C8177A
:1001F00068F520E030E04AE755E4C601B5010E9409
:10020000EA027B018C0120E030E040E85FE30E94DD
:10021000210588231CF481E090E013C020E03FEF2B
:100220004FE757E4C801B7010E94B50418161CF443
:1002300080E090E006C0C801B7010E943601DC01F1
:10024000CB010197F1F7CF5FC91598F2CF911F91BC
:100250000F91FF90EF90DF90CF90BF90AF909F9065
:1002600008954F3F11F4481B4BBB0895EF92FF9246
:100270000F931F937B018C0120E030E040E05FE4AE
:100280000E94EB0488239CF020E030E040E05FEC2B
:10029000C801B7010E948402DC01CB01BC01CD0181
:1002A0000E945705605070408040904804C0C801CB
:1002B000B7010E9457051F910F91FF90EF9008958D
:1002C000A0E0B0E0E6E6F1E00C947E078C017B0153
:1002D0005A01DC018C91823058F0FB019081923000
:1002E00010F4A7010BC1843029F4943009F4A6C09E
:1002F000A80104C19430A9F3923009F4A9C0823056
:1003000081F3F801C280D380FB0162817381F8011F
:100310002481358146815781F7016480758086800C
:100320009780C601861B970B97FDD8C080970CF469
:100330006CC06C157D050CF0ADC0662477244301BC
:10034000F8016181F7018181681709F499C066237A
:1003500009F491C0621A730A840A950AA4019301F0
:1003600057FDC0C0F5011182B60119012A017901BA
:100370008A0139014A0108946108710881089108CD
:10038000FFEF6F16FFEF7F06FFEF8F06FFE39F067D
:10039000F0F4A8019701220F331F441F551F1901C4
:1003A0002A01B601615070406B0179018A0139015F
:1003B0004A01089461087108810891088FEF681656
:1003C0008FEF78068FEF88068FE3980610F383E0AF
:1003D000D5018C9357FC64C0F50124833583468393
:1003E000578373836283A50189C06F5F7F4FD401F8
:1003F000C30181709070A070B070969487947794C8
:100400006794682A792A8A2A9B2A6C157D056CF3E1
:1004100011C00894C11CD11CDA01C901817090700F
:10042000A070B0705695479537952795282B392B96
:100430004A2B5B2BC616D70664F382CFF801918155
:10044000FB018181981709F453CF40E051E056C079
:10045000823009F04DCFDA01F80188E001900D9269
:100460008150E1F7F8018181F70191818923F5013C
:100470008183A50143C0261937094809590970CF5E
:10048000F5016183B601260D371D481D591D19015F
:100490002A019DCF6B0120E030E040E050E050CFDA
:1004A000D201C101B695A7959795879521E030E0D7
:1004B00040E050E02222332244225522282A392AC1
:1004C0004A2A5B2AF50124823582468257820894A3
:1004D000C11CD11CD382C282A50110C09095819508
:1004E0009F4F24CF81E0F5018183B601509540955F
:1004F000309521953F4F4F4F5F4F37CFCA01E2E113
:10050000CDB7DEB70C949A07A0E2B0E0EAE8F2E0DB
:100510000C948C07DC01CB01898F9A8FAB8FBC8F39
:100520002D8F3E8F4F8F58A3BE016F5F7F4FCE013F
:1005300049960E9491068E01075F1F4FB801CE01B8
:100540004D960E949106AE014F5E5F4FB801CE01FD
:1005500001960E9460010E94A905DC01CB01BC014B
:10056000CD01E4E0A0960C94A807A0E2B0E0EBEB8C
:10057000F2E00C948C07DC01CB01898F9A8FAB8F52
:10058000BC8F2D8F3E8F4F8F58A3BE016F5F7F4F63
:10059000CE0149960E9491068E01075F1F4FB80158
:1005A000CE014D960E9491068A8591E089278A871F
:1005B000AE014F5E5F4FB801CE0101960E9460010F
:1005C0000E94A905DC01CB01BC01CD01E4E0A096AD
:1005D0000C94A807A0E2B0E0E0EFF2E00C947E07F4
:1005E000DC01CB01898F9A8FAB8FBC8F2D8F3E8F13
:1005F0004F8F58A3BE016F5F7F4FCE0149960E9477
:10060000910669E070E06C0F7D1FCE014D960E944F
:100610009106FE01319666247724430113012401DB
:100620008981823098F09985923058F420E0918148
:100630008A85981321E02A8769E070E06C0F7D1F9E
:10064000D9C0843059F4923009F45BC020E0918124
:100650008A85981321E02183BF01CCC0943009F42E
:100660004DC0823099F3923009F3ED80FE800F8106
:1006700018852D853E854F855889640153016FE1AA
:1006800070E00CC0220F331F441F551F16950795AD
:10069000F794E7946150704077FD36C0D801C701E8
:1006A00081709070A070B070892BC9F080E090E0EC
:1006B000220E331E441E551E2216330644065506CE
:1006C00010F481E090E0AA2797FDA095BA2F8A0D3B
:1006D0009B1DAC1DBD1D680E791E8A1E9B1EAA0C9B
:1006E000BB1CCC1CDD1C57FFCDCF81E090E0A0E00F
:1006F000B0E0A82AB92ACA2ADB2AC4CF823009F07E
:1007000095CF60E071E076C0228133818B859C8536
:10071000280F391F2E5F3F4FA90160E091818A8524
:10072000981361E06A8B97FE0FC02FC0CA01019732
:10073000AC019C01660C771C881C991C57FC41C0BD
:10074000220C331C441C551C90E0691690E079067D
:1007500090E0890690E4990648F33C8B2B8BD401FA
:10076000C3018F779070A070B07080349105A1059F
:10077000B10581F16D8A7E8A8F8A988E83E0898B9C
:1007800061E170E06C0F7D1F35C02F5F3F4FA90105
:10079000D401C30181709070A070B070892B61F09A
:1007A000569447943794279480E090E0A0E0B0E816
:1007B000282A392A4A2A5B2A969487947794679440
:1007C000C3CF81E090E0A0E0B0E0682A792A8A2ACD
:1007D0009B2AB6CF67FC05C02114310441045104A3
:1007E00049F280E490E0A0E0B0E0680E791E8A1E35
:1007F0009B1EC0CFCB010E94A905DC01CB01BC012F
:10080000CD01E2E1A0960C949A07A8E1B0E0EBE0FC
:10081000F4E00C948607DC01CB01898B9A8BAB8BBF
:10082000BC8B2D8B3E8B4F8B588FBE016F5F7F4FE4
:10083000CE0141960E9491068E01075F1F4FB801BD
:10084000CE0145960E949106FE0131962981223003
:1008500008F45FC03985323010F4B8017BC0818163
:100860009A8589278183243009F455C0223009F400
:1008700052C0343009F454C0323009F458C06B818E
:100880007C818B859C85681B790B2D813E814F81F6
:100890005885ED84FE840F8518892E153F05400785
:1008A000510730F4220F331F441F551F6150704011
:1008B0007C836B8380E090E0A0E0B0E4AA24BB24BA
:1008C00065012E153F054007510740F0A82AB92AB7
:1008D000CA2ADB2A2E193F09400B510BB695A79562
:1008E00097958795220F331F441F551F0097A10529
:1008F000B10539F7D601C5018F779070A070B0703F
:1009000080349105A105B105A9F0A482B582C68203
:10091000D782BF011FC02317E1F760E071E01AC062
:100920001D821E821F8218861C821B82F2CF84E0E9
:100930008983EFCFA7FC05C021153105410551057D
:1009400021F380E490E0A0E0B0E0A80EB91ECA1E3A
:10095000DB1EDBCFCB010E94A905DC01CB01BC0172
:10096000CD01EAE068960C94A207A8E1B0E0EBEBB9
:10097000F4E00C948C07DC01CB01898B9A8BAB8B58
:10098000BC8B2D8B3E8B4F8B588FBE016F5F7F4F83
:10099000CE0141960E9491068E01075F1F4FB8015C
:1009A000CE0145960E9491068981823018F0898592
:1009B000823018F42FEF3FEF09C0B801CE01019645
:1009C0000E940B07282F332727FD3095C901E4E04B
:1009D00068960C94A807A8E1B0E0E1EFF4E00C946D
:1009E0008C07DC01CB01898B9A8BAB8BBC8B2D8B5D
:1009F0003E8B4F8B588FBE016F5F7F4FCE0141966C
:100A00000E9491068E01075F1F4FB801CE014596E7
:100A10000E9491068981823018F08985823018F40D
:100A20002FEF3FEF09C0B801CE0101960E940B07DE
:100A3000282F332727FD3095C901E4E068960C94F0
:100A4000A807A8E1B0E0E7E2F5E00C948C07DC0130
:100A5000CB01898B9A8BAB8BBC8B2D8B3E8B4F8BB9
:100A6000588FBE016F5F7F4FCE0141960E94910665
:100A70008E01075F1F4FB801CE0145960E94910677
:100A80008981823018F08985823018F421E030E0C5
:100A900009C0B801CE0101960E940B07282F332709
:100AA00027FD3095C901E4E068960C94A807ACE0F6
:100AB000B0E0EDE5F5E00C948E07DC01CB01898711
:100AC0009A87AB87BC87BE016F5F7F4FCE010996C7
:100AD0000E9491068981823011F0823028F460E012
:100AE00070E080E090E031C0843039F02B813C81AF
:100AF00037FDF5CF2F3131056CF08A81882329F03D
:100B000060E070E080E090E820C06FEF7FEF8FEF53
:100B10009FE71BC08EE190E0821B930B2D813E81ED
:100B20004F81588504C056954795379527958A95E6
:100B3000D2F78A81882339F05095409530952195D8
:100B40003F4F4F4F5F4FCA01B901E2E02C960C9422
:100B5000AA07A0E0B0E0EFEAF5E00C94840788244F
:100B600099245401DC01FC0124813581468157819F
:100B70008181082F112760E070E08C91823020F491
:100B80006FEF70E04061A4C0843009F464C082302B
:100B900009F463C0211531054105510509F498C0D8
:100BA000FD0182819381FFEF82389F070CF050C0D6
:100BB000A2E8EA2EAFEFFA2EE81AF90A8AE1E8165F
:100BC000F1040CF06BC06B0181E090E0A0E0B0E0BC
:100BD0000E2C04C0880F991FAA1FBB1F0A94D2F7BE
:100BE0000197A109B10982239323A423B523009778
:100BF000A105B10519F0F1E0CF2ED12C04C0569516
:100C0000479537952795EA94D2F7C601AA2797FD0D
:100C1000A095BA2F282B392B4A2B5B2BDA01C9015F
:100C20008F779070A070B07080349105A105B105E8
:100C3000D1F1215C3F4F4F4F5F4F2030E0E03E0746
:100C4000E0E04E07E0E45E0708F161E070E01EC0FE
:100C5000803891053CF06FEF70E020E030E040E03C
:100C600050E036C0BC0161587F4FDA01C9018F776F
:100C70009070A070B07080349105A105B105D1F0DD
:100C8000215C3F4F4F4F5F4F57FD1BC097E056957C
:100C90004795379527959A95D1F71AC020E030E00F
:100CA00040E050E0BBCF27FFC8CF205C3F4F4F4F05
:100CB0005F4FC3CF27FFE8CF205C3F4F4F4F5F4FC1
:100CC000E3CF56954795379527956F5F7F4FDECFDA
:100CD000822E932E942F9F778A2D8078A82EA92A72
:100CE000962F9795992797958A2D8F77A82EA92AC1
:100CF00076956795962F9F778B2D8078B82EB92A99
:100D0000902F9795992797958B2D8F77B82EB92A85
:100D1000D501C401BC01CD01ECE0CDB7DEB70C9428
:100D2000A007CF93DF93FC01DB0140815181228139
:100D3000622F6F7770E0221F2227221F9381892F55
:100D4000880F822B282F3327991F9927991FED0190
:100D500099832115310541F441155105610571054E
:100D6000E1F482E08C9354C02F3F310509F441C077
:100D70002F573040FD013383228383E08C9387E03B
:100D8000440F551F661F771F8A95D1F77064ED01D8
:100D90004C835D836E837F833BC022E83FEFF90184
:100DA000C7E0440F551F661F771FCA95D1F783E030
:100DB0008C93403080E0580780E0680780E4780733
:100DC00078F4440F551F661F771F21503040F901FA
:100DD0004030C0E05C07C0E06C07C0E47C0788F3EB
:100DE000ED01FB83EA83FD014483558366837783AA
:100DF0000FC0411551056105710519F484E08C930C
:100E000007C064FF03C081E08C93C1CF1C92BFCFA9
:100E1000DF91CF9108950F931F93CF93DF93FC0140
:100E2000DB018081823018F09C91923018F461E0EF
:100E300070E05EC08430C1F0843001F1943009F478
:100E400047C0823009F44BC0823009F44EC0923062
:100E5000A9F04181ED0189814817B9F0442389F057
:100E60008FEF9FEFBC0144C0943031F7EB018981D3
:100E7000682F77278181681B71093AC08181882397
:100E800079F781E090E0BC0133C022813381ED012C
:100E90008A819B81821793070CF3281739079CF0EE
:100EA0000481158126813781FD01648175818681E8
:100EB0009781601771078207930780F2061717075B
:100EC0002807390778F4442359F281E090E0DBCF1A
:100ED000FD018181882321F281E090E0D4CF92301E
:100EE00009F0B2CF60E070E003C0ED018981F2CF7C
:100EF000CB01DF91CF911F910F9108952F923F92D7
:100F00004F925F926F927F928F929F92AF92BF9219
:100F1000CF92DF92EF92FF920F931F93CF93DF93C5
:100F2000CDB7DEB7CA1BDB0B0FB6F894DEBF0FBE22
:100F3000CDBF09942A88398848885F846E847D846F
:100F40008C849B84AA84B984C884DF80EE80FD8071
:100F50000C811B81AA81B981CE0FD11D0FB6F894E7
:0C0F6000DEBF0FBECDBFED010895FFCF36
:080F6C0000000000000000007D
:00000001FF
